:020000040800F2
:10000000002000203D230008E11F0008E31F000836
:1000100000000000000000000000000000000000E0
:10002000000000000000000000000000E51F0008C4
:100030000000000000000000E71F0008E91F0008A2
:100040008D230008000000008D2300088D23000888
:100050008D2300088D230008F51F0008FF1F0008EE
:100060000000000009200008192000088D23000866
:100070008D2300088D2300088D2300080000000058
:100080008D23000800000000000000008D23000800
:10009000000000008D2300088D2300088D23000838
:1000A0008D2300088D2300088D23000831200008CF
:0800B0008D2300080000000090
:1000B80010B5064C2378002B07D1054B002B02D036
:1000C800044800E000BF0123237010BD6400002035
:1000D80000000000F4630008044B10B5002B03D0A7
:1000E8000349044800E000BF10BDC04600000000FE
:1000F80068000020F46300080023C25C0133002A72
:10010800FBD1581E7047000002B4714649084900E7
:10011800095C49008E4402BC7047C046002243086F
:100128008B4274D303098B425FD3030A8B4244D3B7
:10013800030B8B4228D3030C8B420DD3FF220902F9
:1001480012BA030C8B4202D31212090265D0030BB8
:100158008B4219D300E0090AC30B8B4201D3CB03AE
:10016800C01A5241830B8B4201D38B03C01A5241F0
:10017800430B8B4201D34B03C01A5241030B8B42F2
:1001880001D30B03C01A5241C30A8B4201D3CB02DD
:10019800C01A5241830A8B4201D38B02C01A5241C2
:1001A800430A8B4201D34B02C01A5241030A8B42C5
:1001B80001D30B02C01A5241CDD2C3098B4201D3DD
:1001C800CB01C01A524183098B4201D38B01C01A5B
:1001D800524143098B4201D34B01C01A52410309D2
:1001E8008B4201D30B01C01A5241C3088B4201D381
:1001F800CB00C01A524183088B4201D38B00C01A2E
:10020800524143088B4201D34B00C01A5241411A54
:1002180000D20146524110467047FFE701B5002061
:1002280000F0F0F802BDC0460029F7D076E7704725
:1002380003460B437FD4002243088B4274D303093F
:100248008B425FD3030A8B4244D3030B8B4228D3E0
:10025800030C8B420DD3FF22090212BA030C8B4206
:1002680002D31212090265D0030B8B4219D300E0A6
:10027800090AC30B8B4201D3CB03C01A5241830B2B
:100288008B4201D38B03C01A5241430B8B4201D3DB
:100298004B03C01A5241030B8B4201D30B03C01A04
:1002A8005241C30A8B4201D3CB02C01A5241830A7E
:1002B8008B4201D38B02C01A5241430A8B4201D3AD
:1002C8004B02C01A5241030A8B4201D30B02C01AD7
:1002D8005241CDD2C3098B4201D3CB01C01A52413E
:1002E80083098B4201D38B01C01A524143098B42C7
:1002F80001D34B01C01A524103098B4201D30B01B0
:10030800C01A5241C3088B4201D3CB00C01A5241D4
:1003180083088B4201D38B00C01A524143088B4299
:1003280001D34B00C01A5241411A00D20146524132
:10033800104670475DE0CA0F00D04942031000D351
:100348004042534000229C4603098B422DD3030AA6
:100358008B4212D3FC22890112BA030A8B420CD3B6
:10036800890192118B4208D3890192118B4204D3DF
:1003780089013AD0921100E08909C3098B4201D35F
:10038800CB01C01A524183098B4201D38B01C01A99
:10039800524143098B4201D34B01C01A5241030910
:1003A8008B4201D30B01C01A5241C3088B4201D3BF
:1003B800CB00C01A524183088B4201D38B00C01A6C
:1003C8005241D9D243088B4201D34B00C01A524143
:1003D800411A00D20146634652415B10104601D3D0
:1003E8004042002B00D54942704763465B1000D35A
:1003F800404201B5002000F005F802BD0029F8D000
:1004080016E770477047C0468446100062468C461F
:100418001900634600E0C0461FB500F0ABFF002896
:1004280001D40021C8421FBD10B500F0EBFE4042C8
:10043800013010BD10B500F09DFF002801DB002041
:1004480010BD012010BDC04610B500F093FF002874
:1004580001DD002010BD012010BDC04610B500F020
:1004680015FF002801DC002010BD012010BDC0468A
:1004780010B500F00BFF002801DA002010BD0120A4
:1004880010BDC0469E2110B5C905041C01F00AFB29
:10049800002803D1201C00F0EFFA10BD9E21201C7B
:1004A800C90500F045F900F0E7FA80231B069C46D1
:1004B8006044F2E7F0B54F464646D64643025B0A2B
:1004C8004500C0B599460F1C2D0EC60F002D00D152
:1004D80088E0FF2D00D18DE08022DB00D2041A4392
:1004E8000023914698469A467F3D7C027B00640A29
:1004F8001B0EFF0F002B68D0FF2B21D08022E400B9
:10050800D204144342467F3B5B1900215D1C0A2A32
:100518002EDC7E404246022A23DC013A012A00D919
:10052800BDE002296ED001292CD100200022C0058F
:10053800F60710433043E0BCBA46B146A846F0BDC2
:100548002B00FF33002C65D00322414611433200B3
:10055800013588467A40FF350A2900DDD8E01600C3
:100568000321404601228240A620C000024220D03A
:100578005346022B46D0032B00D1BBE051464C46D4
:100588000129D2D02B007F33002B70DD620704D005
:100598000F222240042A00D00434220103D5634BE1
:1005A8001C402B008033FE2B2CDCA201520AD8B24F
:1005B800BDE790208000024227D1B938FF381042A9
:1005C8006DD03E00A1468A46D2E7002C41D10123D6
:1005D80042461A4390462B00424601215D1C0A2AD6
:1005E80097DDC5E7002B26D104239846033B002559
:1005F8009A467AE7002B18D108239846063BFF2530
:100608009A4672E7FF20002291E780220026FF2009
:10061800D2038CE741460222013511438846FF3553
:100628000A29A5DC02217E4074E70C239846093B81
:10063800FF259A4659E7180001F03EFA4A46431F3B
:1006480076259A4000236D42914698469A462D1A7F
:100658004BE7200001F030FA4246431F9C402B1A1A
:10066800763B00215D1C0A2A00DC52E780E7012264
:10067800D31A1B2B00DD58E79E352200AC40DA4028
:10068800631E9C412243530704D00F231340042BBD
:1006980000D00432530137D50120002247E7210C4E
:1006A8004A462404240C2700100C1204120C44435C
:1006B8005743484351433A0C09195218944203D9F5
:1006C800802149028C4660443F0411043F0CC9193B
:1006D8008C01671EBC41120C890E12180C43920142
:1006E800144312010ED5012362081C40144349E744
:1006F8003E00A14680224B46D2031A435202FF20F5
:10070800520A14E71D003DE792010020520A0EE745
:100718000F29EDD180224B46D2031342EAD014426E
:10072800E8D13E00FF20224301E7C046FFFFFFF764
:10073800F8B54746CE464E0243024500720AC40F3A
:10074800480080B594465F0A2D0E9B09000EC90F1C
:10075800B609FF2824D0012251402A1A8C420FD012
:10076800002A00DC6AE1002835D1002E00D1A2E081
:10077800511E012A00D124E1FF2A21D00A002FE0CE
:10078800002A00DC67E100285ED0FF2D18D0802108
:10079800C9040E431B2A00DC76E02A00013332E04C
:1007A8002A00FF3A9146002E42D08C4255D04A4644
:1007B800002A00D19CE0002D00D177E00C00330026
:1007C800DB08002B00D16EE08022D20313435B02CA
:1007D800FF205B0A24E0FF2DF2D08021C9040E43DC
:1007E80001211B2A08DC31002020D140821A9640C2
:1007F8003200501E824111435B1A5A0160D407210E
:100808002A00194057D00F211940042900D0043379
:10081800590150D5501CFE2A45D09B01C0B25B0A35
:10082800C0051843E4072043C0BCB946B046F8BD2C
:10083800012251408C42BAD14A46002A10D0002DDC
:1008480000D198E00023BBE7002E34D0511E012AC6
:100858006ED0FF2AB4D00A009CE7002A00D088E0B6
:10086800FE206A1C104200D092E0002D00D0A4E0C7
:10087800002B00D1CBE0002E00D0CAE00022DB081C
:100888005B025B0AD0B2CBE731002020D140821A4C
:1008980096403200501E82410A439B185A01AED539
:1008A8006A1CFE2D4AD1FF200023B9E7FF22002B46
:1008B8004BD10C003300DB08FF2A00D181E7DFE7CA
:1008C8009F01BF09380001F0F7F8053887408542D5
:1008D80021DC3B002021421B0132D3408A1A974079
:1008E8007A1E974100223B43590700D08BE78FE7D8
:1008F800FE206A1C104212D1002D52D1002B7CD050
:10090800002EBBD09A1B500100D48BE0012400229A
:10091800F31A0C40E8E7564B2A1A3B40E4E79F1BC2
:100928007A0146D4002FCDD100240020002377E798
:100938009B1901250132590100D460E701214D4876
:1009480019405B0803400B43CEE7571E012A5AD0D3
:100958000C00FF2A33D001221B2F07DC2021C91BE2
:100968001A008B40FA40591E8B411A430500B31AEE
:1009780043E7002D23D1FF22002B9BD0511E012AD3
:10098800D6D0FF2A1BD01B292CDD0200731C3AE7A6
:10099800FF2A88D09B195B08590700D033E7DB088A
:1009A8006EE7002B10D1002E43D0012433000C40F9
:1009B80006E70124F71A0C4084E7002B04D1330022
:1009C800FEE601259B1B18E7002E00D1F8E68022E1
:1009D800D203974204D3944502D2012433000C4039
:1009E800DB08F1E61A002025CA40691A8B40591E17
:1009F8008B41134305009B1950E7002E94D0012426
:100A080033000C403AE70C000125F31AF5E63300F1
:100A180034E79B1900225901C1D5154A1340DB0858
:100A280001222DE7002A00D17EE713000022DB080F
:100A380026E780230024FF20DB03F1E6002A00D10B
:100A480056E7471B3A00002D00D130E78022D20438
:100A58000C0013437FE7002A00D101E7411B002D5A
:100A680001D10A0088E78022D20413438BE7C046ED
:100A7800FFFFFFFBFFFFFF7D41024200C30F490A52
:100A88000020120E7E2A03DD9D2A02DD094A9818ED
:100A98007047802000040143952A07DC9620821ABB
:100AA800D1404842002BF3D10800F1E7963A914033
:100AB800F7E7C046FFFFFF7F70B5041E0ED000F0B9
:100AC800FBFF9E2301001B1A962B0CDC08282FD055
:100AD80008398C406402640AD8B201E0002000247E
:100AE800C005204370BD992B16DC421F052800D095
:100AF8009440220010480240650709D00F252C4079
:100B0800042C05D00432540102D59F2302405B1AFD
:100B18009201540AD8B2E3E7020020001B32904049
:100B28000200501E82410520401AC4401443E0E7E9
:100B380064029620640AD3E7FFFFFFFBF0B557462F
:100B48004E464546DE46E0B583B0009001910C0361
:100B58004F00CE0F610A009C1D03640F0C430099DF
:100B680000920193C80059004B0D9946009A019BC9
:100B78006D0AD90F530F2B439A46009B7F0DDA005D
:100B880094464A46B046BA1A8E4200D1B0E0002ACE
:100B980000DC78E04946002900D1E9E0C9498F42E4
:100BA80000D195E10125382A16DC80215346090435
:100BB8000B439A461F2A00DDE7E1202155468B1A90
:100BC80061469D40D1400D43614699404B1E994175
:100BD8005346D3400D43E41A451BA8428041404286
:100BE800241A230200D40FE16402640A002C00D105
:100BF80039E1200000F060FF0300083B20212800B5
:100C0800CA1AD0409C4002009D4022439F4200DD0A
:100C180073E1D81B0130091A2C008D40C4406B1EAB
:100C28009D411300C2408B402543002714001D43FB
:100C38006B0709D00F232B40042B05D02B1DAB428B
:100C4800AD416D4264191D00230200D42DE19D4A77
:100C58000137974200D1D3E046469B49ED08214031
:100C68004A072A437C054D022D0B640D24052C43AD
:100C7800F60734431000210003B0F0BCBB46B2466F
:100C8800A946A046F0BD002A00D184E04A46D21BFE
:100C9800002F00D06DE12500054300D127E1561E45
:100CA800012A00D13BE2874DAA4200D16AE2012520
:100CB800382E12DC32001F2A00DDF8E1202625003C
:100CC800B61A07005346B040D440B540D740461E38
:100CD800B0411B1B9A463D4305436246551BAC4534
:100CE8009241534652420E004F4688469C1A78E776
:100CF800002A00DC8EE04946002975D1614653463A
:100D0800194300D1F6E0511E012A00D191E16D4D41
:100D1800AA4200D1DCE00125382914DC0A001F2A88
:100D280000DDA2E120215346891A8B401D0063464D
:100D3800D3401D4363468B4019004B1E99415346CF
:100D4800D3400D43E4182D188542804140422418B1
:100D5800230259D55B4B01379F4251D001215A4B91
:100D68006A081C4029400A43E507154364085FE701
:100D780061465346194300D1BCE0511E012A00D1F7
:100D880064E1504DAA4200D16AE10125382900DD0D
:100D980022E70A000EE74D4A7D1C154200D0D0E03C
:100DA80025006246534605431A43002F00D037E119
:100DB800002D00D1A8E1002A00D16AE16346C51AD6
:100DC8005346E21AA8429B415B42D31A1A0200D446
:100DD80003E263461D1AAC459241534652421C1B1E
:100DE8000E008846A41A23E736498F4270D00125A1
:100DF800382AA8DC8021534609040B439A468EE71B
:100E08003C000025002231E707232B40002B00D0AF
:100E180010E793E0002A74D04A46D21B002F00D175
:100E2800C7E02849894500D185E10125382A12DC27
:100E3800802109040C431F2A00DDABE12021250095
:100E4800891A070088408D40D740411E8841D44008
:100E58003D430543A244654465459241524252448C
:100E680014004F4674E7280000F026FE03001833EC
:100E78001F2B00DCC2E62A00083882409F4200DDB2
:100E8800A9E0DB1B581C1F2800DCACE115001F3B48
:100E9800DD40202805D040231B1A9A40531E9A4152
:100EA8001543072300272B40B0E7ED08054B6207E1
:100EB8002A43E4089F420FD02403250B7C05640DC8
:100EC800D4E6C046FF070000FFFF7FFFFE070000D3
:100ED800C00862070243E4081300234300D186E1F7
:100EE80080252D0325432D03C34C2D0BBEE66046FC
:100EF80054460E001700C508D8E7C04CFF1A144026
:100F080096E6BF4A791C11426BD122000243002F9A
:100F180000D0DBE0002A00D12DE1624653461A4397
:100F280000D1B6E06346C51885428041544440422A
:100F38002418230202D50F00B04B1C403A002800A9
:100F4800D8E76246851AA8429241534652429146D2
:100F5800E31A1A004B46D21A130091461A0254D4C7
:100F68004A464C462A4300D040E600260024002585
:100F78007CE6A14DA94500D190E00125382A00DD85
:100F8800ABE680252D042C4395E611005546203903
:100F9800CD40A946202A06D0402153468A1A9340BC
:100FA80062461A43944665466B1E9D414B461D4357
:100FB80012E62100014300D1C4E0511E012A00D1EC
:100FC800FBE08D4DAA4200D1B5E00125382900DDAE
:100FD80041E70A002FE7894CFF1A14406207E4082A
:100FE8006AE7854A914200D1E3E06346C21882422B
:100FF80080412300404253441B18DD075C08072347
:10100800520815430F002B4000E763461D1AAC45F4
:101018009241534652421C1B0E008846A41AE5E52D
:10102800002D00D091E0002A38D180240026240326
:1010380056E76346C5188542804154444042241807
:101048000127230200D4DFE6022787E66346C51A94
:10105800A842804153464042E41A0127241AC0E5B9
:101068006207C0080243E40836E7110053462039F6
:10107800CB409946202A06D0402153468A1A9340ED
:1010880062461A43944665466B1E9D414B461D4376
:1010980059E66207C0080243E4080DE753465A07B9
:1010A8006346D80853460E000243DC0814E71500CF
:1010B8002600203DEE40202A03D04025AA1A94405D
:1010C8002043421E90410500354306E6002A7CD0A5
:1010D80062465346C0081A4300D1FAE66207104335
:1010E8008022E4081203144208D0D908114205D11D
:1010F8006346D80853460C005B071843420FC000EC
:10110800C00852070243E7E6002A00D12DE76346EC
:10111800D80853465A070E000243DC08CCE663465B
:101128001D1AAC459241534652421C1B0E0088467C
:10113800A41A013755E56346D90853465A070A43A6
:10114800DC08C9E660465446D4E6C008002A00D147
:10115800BFE6620710438022E40812031442CDD090
:10116800DD081542CAD16346D80853465B070E000E
:101178002C001843C2E76346D90853465A070A4366
:10118800DC0899E66346D80853465A070E0002431E
:10119800DC08A1E6110027002039CF40202A03D01F
:1011A80040218A1A94402043421E904105003D4345
:1011B80051E60C000025002258E560446045924144
:1011C800544452420500A4183AE753465A07634666
:1011D800D90853460A43DC087EE61A001C002A4355
:1011E80000D0ABE6C1E620210025091A19E5002246
:1011F8000025014C3AE5C046FF070000FFFF7FFFCE
:10120800FE070000F0B55746DE464E464546E0B5B7
:101218000D000400E80F83460903D80F090B824626
:1012280019488C461F0369005E00490D3F0B760D77
:10123800814218D086420FD00120B1420DD1BC4561
:101248000BD1944209D1D3451CD0002905D1604661
:101258002043431E984100E00120F0BCBB46B24643
:10126800A946A046F0BD01208E42F6D16146394319
:101278000F0017432743F0D15B465246981A431E86
:101288009841EAE70020E8E7FF070000F0B5574675
:101298004E464546DE46E0B50D000F03390B83B0D8
:1012A8000400804601915800E90F314F400D8C46EB
:1012B8006E00190382469146760D090BD80FBE427F
:1012C8001FD0BA450FD0002E2FD15546019E34436A
:1012D800002D27D10A433AD0002C45D100281AD135
:1012E8000120404217E011433BD1002E02D1019F5B
:1012F8002743F3D0844509D16346002BF0D06046DC
:1013080009E0019F27432CD1B24524D0634602202F
:10131800013B1840013803B0F0BCBB46B246A946B1
:10132800A046F0BD002CD9D0E4E75446002CEDD0FF
:101338008445EBD15645E9DCDEDB019B8B42E5D8E1
:10134800DAD1C845E2D80020C845E4D2D4E7002065
:10135800002CE0D0DAE7114303D18445D6D1002030
:10136800D9E702204042D6E78445E6D0CEE7C0461A
:10137800FF070000F0B557464E464546DE46E0B545
:101388000D000F0304008046E80F390B844683B034
:101398005800304F400D01911E0369008246914666
:1013A800490D360BD80FB94220D0BA450FD00029C5
:1013B8002BD101990C435146002937D1324338D0FB
:1013C800002C44D1002819D10120404216E01643D0
:1013D80013D1002902D1019F2743F3D0844520D09F
:1013E80063460220013B1840013807E0019F27436C
:1013F80003D18A45F4D116431FD0022003B0F0BCB4
:10140800BB46B246A946A046F0BD5446002CE7D0DC
:101418008445E5D15145E3DC03DB019BB342DFD8CA
:101428000FD06346002BCFD06046E7E7002CC9D029
:10143800D4E70020002CE1D0D2E78445D0D10020A9
:10144800DCE7C845CCD80020C845D7D2E9E78445B1
:10145800E3D0C5E7FF070000F0B55746DE464E4625
:101468004546E0B51F000B031B0B16009A46CA0F32
:101478004B000400934687B05B0D00D1D5E0BB4A12
:10148800934200D1F8E05146420FC9000A43802137
:1014980009041143C2009146B54A8A469D180023A3
:1014A800984602933C037B00FA0F3000240B5B0D37
:1014B800009200D196E0AD4A934231D0720FE40019
:1014C8002243802424041443A94AF0009446634428
:1014D8005B195A1C0192424600260A2A42DC5A46E7
:1014E80000994A4093464246022A32DC013A012AD0
:1014F80000D949E1022E00D1CAE0012E3DD10023D6
:101508000024002210005A461B052343D207134328
:10151800190007B0F0BCBB46B246A946A046F0BDCC
:10152800924B2643EB18002E00D1BBE00322414624
:1015380011435A46884600994A40802109018C4641
:1015480029006144019141460A2900DD33E29346AE
:101558000326424601279740A6213A00C9000A40BF
:101568000F4231D0029E022E00D135E2032E00D167
:10157800D2E154464846012EC1D0019A7D4B94468B
:101588006344002B00DCC0E0420709D00F22024070
:10159800042A05D0021D82428041404224181000CE
:1015A800E20106D5744B019A1C4080239446DB0067
:1015B8006344724A93426BDC6207C00864025B05AD
:1015C8000243240B5B0D9DE7902189000F4263D1F4
:1015D80088223A4200D1D7E0009BA2469B4681462A
:1015E8000296BFE72300334300D17FE0002C00D1EF
:1015F800ADE1200000F060FA020003000B3A1D2064
:101608001900821A30000839D0408C400443300059
:1016180088405B4AEB1A944663445A1C019242463E
:1016280000260A2A00DC5AE79CE7534603439946FA
:1016380054D05346002B00D177E1504600F03CFAD5
:101648000B235B429C460200844411005046083933
:1016580088401D23804660461B1A2000D84003009E
:10166800404603439A4623008B4099460023444D45
:101678009846AD1A029315E752460243914626D181
:1016880000221D000223924608329046029309E781
:1016980000240022354B35E7002380249B46240391
:1016A800324B2FE702224146114380221201944611
:1016B8002A006244884601920A2900DD52E75A4608
:1016C8000020009904004A40934602260BE70C22AA
:1016D8001D000323814690460293E3E600239A46C1
:1016E80004339846033B00250293DBE64246013368
:1016F8001A432B0090465A1C0192424600240020AF
:1017080001260A2A00DCEAE62CE70122D21A382A46
:1017180000DDF4E61F2A00DC2AE11F214942CB1A2A
:101728002100D9400B00202A05D0164A019D944675
:101738006544AC402043421E9041184307231900DA
:101748000024014003420CD00F230340042B00D196
:1017580040E1031D8342A44118006442610764020A
:10176800240BC20800230A43CCE6C046FF0700004A
:1017780001FCFFFFFF030000FFFFFFFEFE07000064
:101788000DFCFFFF3E04000049464A460904090CC7
:101798000D00160C020C0004000C4543AC46050075
:1017A8007543A84615000F007543009202952A005C
:1017B800009D6F4365462D0CA94647444F44B845E4
:1017C80005D91500802252029046454402953D0CE9
:1017D800039565462D043F042D0CAC463D00654439
:1017E8000495250C2404240CAC4625007543A84612
:1017F80065460F006943414489466743390C4944AB
:101808006E43884503D980225202904646440D0C07
:10181800A846350045440595039D3F04A8463F0C5E
:101828000904C91988444546039555462E04360CC3
:101838002F0C35004543784381463800A8462D0CC7
:10184800AA46009A504372434A445244914503D9E8
:1018580080256D02A9464844150CA94645462D0425
:101868002D0CA84665467D43120448449044A94679
:101878003200654662436E437C43170C3619BF1924
:10188800BC4203D980246402A446E144029C039E1E
:10189800A446059D66448E428941AC4612043C0428
:1018A800120CA2186244494254184644A4464645BC
:1018B800A44182466442A046AA4292418C4589418D
:1018C800E244D044494252420A43A045A4418245D9
:1018D8008941644249420C4341463F0CD2191219CE
:1018E800CC0D049970020843411E884141464A4480
:1018F800F60D52023043490214430843D20135D54C
:101908000122430802401343E0071843640834E601
:10191800009BA2469B4681468024534624031C43D1
:1019280024034A462E4B240BECE500F0C5F815239A
:101938009C4684440200634620321C2B00DC84E66B
:10194800002399462300083883409A468EE600F023
:10195800B3F802000300153220331C2A00DC4EE6DF
:1019680002003400083A0020944052E6019304E64D
:101978001C4B21009C460300019DD3406544A940AF
:1019880019430300AB40581E834119430800D44053
:101998004B0709D00F230B40042B05D00B1D8B429E
:1019A8008041404224181800230200D4D6E60123BF
:1019B80000240022A6E50F29AAD1802352461B0342
:1019C8001A42A9D01C42A7D11C43009B02009B4687
:1019D800034B97E50024C1E60024014B220091E562
:1019E800FF0700001E04000070B5002816D0C317BA
:1019F800C5185D40C40F280000F05EF8104B1B1A94
:101A08005B055B0D0A2814DC02002E001532964097
:101A18000B22121AD5402D032D0B03E000240023BE
:101A2800002500261B052B43E4072343300019003B
:101A380070BD0B3885402D0300262D0BF2E7C046FC
:101A48001E040000844608006146FFE71FB500F049
:101A5800C9F8002801D40021C8421FBD10B500F004
:101A680049F84042013010BD10B500F0BBF800281D
:101A780001DB002010BD012010BDC04610B500F0EC
:101A8800B1F8002801DD002010BD012010BDC046BE
:101A980010B500F057F8002801DC002010BD012027
:101AA80010BDC04610B500F04DF8002801DA00203E
:101AB80010BD012010BDC0461C2101231B04984203
:101AC80001D3000C10391B0A984201D3000A0839C7
:101AD8001B09984201D30009043902A2105C40187E
:101AE8007047C04604030202010101010000000022
:101AF8000000000070B542004E024C0045026D0A1D
:101B0800120EC30F760A240EC90FFF2A10D0FF2C1D
:101B18000CD00120A2420AD1B54208D18B420FD085
:101B2800002A04D12800431E984100E0012070BD1E
:101B38000120FF2CFBD13543F9D14B401800F6E7C3
:101B48000020F4E730B5420044024D02C30F4800BC
:101B5800640A120E6D0A000EC90FFF2A19D0FF2859
:101B68000BD0002A1ED100280BD1002D27D0002C25
:101B780034D100292FD0080030BD002D28D1002AEB
:101B880001D1002CF5D08B4207D1002B23D01800AF
:101B9800F2E7002C1CD1FF2814D0581E022318404D
:101BA8000138E9E70028F8D08B42F6D18242F4DC0C
:101BB800EBDBAC42F1D80020AC42DDD2E5E7002CEB
:101BC800DAD0EAE7002D03D18B42E6D10020D3E733
:101BD80002204042D0E701204042CDE78B42E8D0C6
:101BE800DBE7C04630B5420044024D02C30F48004F
:101BF800640A120E6D0A000EC90FFF2A1AD0FF28B8
:101C08000ED0002A1ED100280ED1002D2AD0002C7B
:101C18000CD08B421DD0581E02231840013810E00A
:101C2800002D0DD1002A20D1002C1ED1002923D04F
:101C3800080006E0002C03D1FF28ECD1002D17D0B6
:101C4800022030BD0028E6D08B42E4D18242E2DC9B
:101C580004DBAC42DFD80020AC42F2D2002B0BD020
:101C68001800EEE7002CECD0D5E78B42D3D1F5E78E
:101C780000208B42E5D0CEE701204042E1E7C04694
:101C88001FB50C22002101A804F07AFB8022184C11
:101C9800184B120622610422236080236261033AF2
:101CA8001B03A276E2612200636000232C321370CA
:101CB80007226263220020003C32A360E360238392
:101CC8006362A36223631370E36400F0AFFB002830
:101CD80001D000F067F9084B20000193012301A906
:101CE800029300F00BFD002801D000F05BF91FBD46
:101CF800DC000020002401400200000470B505004B
:101D08008EB01422002103A804F03AFB1822002107
:101D180008A804F035FB264B2A689A4245D180234F
:101D2800DB010893802308A81B060C9301F022FF0F
:101D3800002801D000F036F980211E4B49031A6CA7
:101D4800A0200A431A641A6C00260A400121019255
:101D5800019A5A6BC0050A435A635B6B05960B40A0
:101D68000293029B022303935B1803A9049301F0D7
:101D780067FA114C114B20002360052363607B3305
:101D88002361803363618023DB00A3612023E36147
:101D980080235B01A660E660236200F0BDFFB042CD
:101DA80001D000F0FFF82C65A5620EB070BDC046EA
:101DB800002401400010024080000020080002407A
:101DC80007B501210C4B09209A6B0A439A639B6B58
:101DD80000220B4001934918019B00F003FF0920E2
:101DE80000F02AFF002202210A2000F0FBFE0A2050
:101DF80000F022FF07BDC04600100240F0B50227E0
:101E08000125A02689B01422002103A804F0B8FAFD
:101E1800394BF6055A6B30003A435A635A6B3749C7
:101E28003A400192019A5A6B00242A435A635B6B29
:101E38002A002B400293029B01F02CFB3000002269
:101E4800202101F027FB2A0029002D4801F022FB60
:101E58000423300003A9039304950594069401F024
:101E6800EFF908230393C42330009B0303A90493C9
:101E7800059401F0E5F92023300003A903930495A4
:101E88000594069701F0DCF94023300003A9039379
:101E98000494059401F0D4F9802303938823300037
:101EA8005B0303A90493059401F0CAF903A9144834
:101EB800039504950594069401F0C2F9C0235B01CB
:101EC80003931123300003A904930594069701F0A6
:101ED800B7F922003900062000F084FE062000F041
:101EE800ABFE22003900072000F07CFE072000F03E
:101EF800A3FE09B0F0BDC04600100240041800005F
:101F08000004005010B592B03422002105A804F056
:101F180037FA1022002101A804F032FA802080004C
:101F280001F0DAFA0A230593F6330893002309939C
:101F38000E9308330F9380239B0240221093802333
:101F480002240A929B053F3A05A80B920C940D9423
:101F5800119301F0EDFA002801D072B6FEE70723CD
:101F680003900490210001A80193029401F040FD20
:101F7800002801D072B6FEE712B010BD10B500F00F
:101F88002BFAFFF7BFFF04F00DF9FFF737FFFFF754
:101F980017FFFFF775FE00F0B7F800F0F1F803F04F
:101FA8004BFFFEE772B6FEE701210A4B82B01A6CBE
:101FB8000A431A641A6C0A4080210092009ADA6B6C
:101FC80049050A43DA63DB6B0B400193019B02B0BE
:101FD8007047C04600100240FEE7FEE770477047B2
:101FE80010B500F00DFA04F00FF910BD10B5082077
:101FF80001F05EFA10BD10B5802001F059FA10BD4D
:1020080010B5024800F0E2FF10BDC0468000002075
:1020180010B5034800F0DAFF024800F0D7FF10BD02
:10202800E80100208C01002070B5134C200002F05C
:1020380001FB200002F042FA102223680F4DD969F3
:10204800114212D01A620E4A1378002B0DD10D4B93
:102058000D481B68596880235B425B1ADBB213701A
:1020680012782900D2B204F0B7F9290080222000A2
:1020780002F020FF70BDC046440200206706002021
:10208800E7060020E80100206705002070470000EF
:10209800084B026882B09A4209D18021064B090296
:1020A8001A6C0A431A641B6C0B400193019B02B023
:1020B8007047C046002000400010024010B50400E0
:1020C80086B01422002101A804F05AF90C4B2268AA
:1020D8009A4213D101210B4BA0205A6BC0050A4329
:1020E8005A635B6B0B400093009B102301930E3BDC
:1020F800029301A90233059301F0A2F806B010BDBE
:10210800002000400010024010B588B01C220021B9
:1021180001A804F035F9174C174B184A236002231D
:10212800636000232000A360E2602361A36101F0E3
:1021380051FF002801D0FFF735FF200001F074FFA0
:10214800002801D0FFF72EFF60230193FA23002215
:102158009B00200001A902930392059201F0CAFF97
:10216800002801D0FFF71EFF2000FFF7A7FF08B0E7
:1021780010BDC0464001002000200040E7030000D9
:1021880010B5184B184C0C22236096239B016360F2
:1021980000232000A360E36023616261A361E3611F
:1021A80023626362A36202F0FBFD002801D0FFF7FF
:1021B800F9FE0021200002F0F5FE002801D0FFF70B
:1021C800F1FE0021200002F00DFF002801D0FFF7EA
:1021D800E9FE200002F0C8FE002801D0FFF7E2FE69
:1021E80010BDC046003801404402002070B506000A
:1021F8008EB01422002103A804F0C2F8182200218E
:1022080008A804F0BDF8334B32689A4260D1012324
:1022180008A8089301F0AEFC002801D0FFF7C2FE21
:1022280080212D4BC9011A6C00250A431A641A6CC7
:102238002A480A400192019A0222596B11435963B4
:102248005B6B03A913400293029BC0230492039380
:1022580005950695079500F0F3FF214C214B2000CA
:102268002360322363604E33236180235B01A560C2
:10227800E5606561A561E561236200F04DFDA84256
:1022880001D0FFF78FFE331DDC67A662164B174C93
:102298008022236033236360233BA3600023E36031
:1022A8006361A361E361802320005B0122612362F3
:1022B80000F032FD002801D0FFF774FE1B20002239
:1022C8000121F467A66200F08DFC1B2000F0B4FC2D
:1022D8000EB070BD003801400010024000040050EC
:1022E800E80100201C000240300002408C01002060
:1022F8000C4B026810B504009A4212D10A4A0B49E5
:10230800136C0B480B401364C02101F04BF8231DDC
:10231800D86F00F05BFDE06F00F058FD1B2000F067
:1023280097FC10BD0038014000100240FFBFFFFFBE
:10233800000400500D488546FFF7A8FE0C480D49DB
:102348000D4A002302E0D458C4500433C4188C4208
:10235800F9D30A4A0A4C002301E013600432A2426E
:10236800FBD304F015F8FFF709FEFEE70020002074
:102378000000002064000020B4640008640000200D
:1023880070070020FEE7000070B5104B05001978B3
:10239800002901D1012070BDFA208000FDF7BEFEA2
:1023A8000B4C01002068FDF7B9FE00F061FC041E2B
:1023B800F0D1032DEED8020001202900404200F0A0
:1023C80011FC044B20001D60E5E7C0460400002016
:1023D80000000020080000208023084A5B001168E4
:1023E80010B50B4303201360FFF7CEFF041E03D183
:1023F800FFF7DAFD200010BD0124FBE700200240B2
:10240800034A044B11681B785B1813607047C04679
:10241800D802002004000020014B18687047C0460D
:10242800D802002080684007C00F70470023F0B52D
:1024380085B004000393984200D1F0E0856D9D4279
:1024480005D1FFF75BFC23005433E5651D7080233D
:1024580025685B05AA681A4200D1A7E00022AB688C
:102468000192DB0008D410230126A26D01961343C4
:10247800A365E36D3343E3652800FFF7D3FF10221C
:10248800A36D1340034300D0CCE0A26D674B2069D5
:102498001A400633FF331343A365AB68DB0761D4E7
:1024A800276BE1687B1E9F41A368A27E0B43217EB8
:1024B8003F0389030B43617EC9030B4351030B435D
:1024C8009C46002800DB86E0410049082300664658
:1024D8002C331B785B0033433B430B43611CC97FA0
:1024E800012905D1002A00D078E080225202134346
:1024F800626A002A05D0E02149000A40A16A0A431D
:102508001343EA684A490A401343EB6023006268B0
:102518003C33E16C1B78970FBF079C463943012B6E
:1025280008D1236C666C33430B43A16C0B436146A3
:102538003B4319432B693F4F3B400B4380212B61A1
:1025480053005B08C9058B420CD080231B069A42B6
:1025580008D03949394F0B683B40F027BF033A4050
:1025680013430B60072170276B69626B8B4313431E
:102578006B616969A36BB9431B010B436B6100284D
:1025880034D11023A96A5B420B43AB6207216B6904
:102598000B409A4239D10023E365A26D03339A4375
:1025A800023B1343A365019805B0F0BDAA6824490E
:1025B8000A401343AB60234B23491868FDF7AEFD6F
:1025C800013040000390039B002B00D146E7039B9A
:1025D800013B0393F7E78021890377E72022A76D62
:1025E8003A43A265E26D1143E16581E780239B03CD
:1025F8009842CBD11C21AB6AE369013B9B000B409D
:102608002C3999400B00216EBEE71223A26D9A4324
:10261800023B1343A3650123E26D1343E3650123E2
:102628000193C0E7A36D1A43A265F8E7FDFEFFFF1B
:102638000102FEFF02FCFF1F08270140FFFFC3FF46
:10264800E8FFFF6F00000020400D0300704770474F
:1026580010B5806AFFF7FBFF10BD70474023806A02
:1026680010B5826D134383650423C26D1343C3659C
:10267800FFF7F3FF10BD0000502370B5846AA26D08
:102688001A422DD1A26DB133FF331343A365C02382
:1026980025681B01EA681A4215D1A37E002B12D1C6
:1026A8002B681B070FD52800FFF7BCFE00280ED1AA
:1026B8000C226B6893436B60A26D0F4B1A40043376
:1026C800FF331343A3652000FFF7C0FF70BD20232D
:1026D800A26D1343A3650123E26D1343E365F2E79B
:1026E800A36DDB0603D52000FFF7B7FFEEE7236DE8
:1026F8005B6B9847EAE7C046FEFEFFFF0023F0B594
:1027080085B003930300009154331A780400022023
:10271800012A4CD0012227691A7025682800FFF782
:1027280081FE002800D0E9E0009B04225B6880213C
:102738009C4697436246009B09061B68022A00D103
:10274800B0E05A03520B8F4233D1A96A0A43AA62F6
:10275800009A6869926819026B4E0A4032408843B1
:1027680002436A61002B1EDAE021684A684815684E
:1027780049042940834200D07EE0802000040542BD
:1027880011D11368634D2B400B431843624B106003
:1027980018686249FDF7C2FC431C0C20584303909B
:1027A800039B002B64D1002000235434237005B010
:1027B800F0BD1F2167460F401039B940CE4301963E
:1027C800266E8E433100002A12D1980E1F32104017
:1027D800B840624608439208E169013220668A429D
:1027E800B6D8A96A01989A00120FBA400140ADE71D
:1027F80001221342ECD1921801201342E8D11000B3
:1028080002321342E4D101301A07E1D40130DA066A
:10281800DED401309A06DBD401305A06D8D4013010
:102828001A06D5D40130DA05D2D401309A05CFD4AE
:1028380001305A05CCD401301A05C9D40130DA0464
:10284800C6D401309A04C3D401305A04C0D401302C
:102858001A04BDD40130DA03BAD401309A03B7D4CC
:1028680080221800D20210401342B1D01220AFE7E4
:10287800039B013B039393E7294883420BD18020B4
:102888004004054200D08EE71368224D2B400B43CD
:102898001843106087E72348834200D083E78020ED
:1028A800C003EEE78F4204D1AA6A5903490B8A4351
:1028B800AA62002B00DB76E7144A154811688342A8
:1028C80008D1A02310685B040B40124901400B4358
:1028D800136068E71248834203D1C02310681B04C1
:1028E800F2E71048834200D05DE7C0204004136837
:1028F8000140084803401943116054E72023A26DA2
:1029080001201343A3654FE700FFFF070827014095
:10291800001000B0FFFF3FFE00000020400D030044
:10292800004000B8002000B470B505680400280015
:10293800FFF778FD002801D1002070BDAB689B0728
:1029480005D4AA680F4B1A4010231343AB60FFF756
:1029580063FD0426050023689B683342ECD0FFF72B
:102968005BFD401B0228F6D923689B683342F2D0EE
:1029780010230120A26D1343A365E36D0343E365B0
:10298800DBE7C046E8FFFF7F0023F7B50268019345
:10299800916801330400194201D00020FEBD9068FF
:1029A8002249084208D01022A16D0A43A265E26DAF
:1029B80013430120E365F1E791681D4F39400B434C
:1029C80093601C4B1B681B0221D4637E012BE4D04F
:1029D800FFF722FD01250600226813682B42DCD18F
:1029E80093682B4203D193683B402B439360FFF7D6
:1029F80013FD801B0228EFD923681B682B42EBD1FB
:102A08001023A26D1343A365E36D2B43D1E70A4B53
:102A18000A491868FDF782FB01300190019B002BE1
:102A2800D3D0019B013B0193F8E7C0461700008013
:102A3800E8FFFF7F0827014000000020400D030049
:102A4800F7B50568040028000E000192FFF7EAFCBC
:102A5800022300283FD1270054373A78012A3AD078
:102A6800013B3B70EA681A420CD1AA681A4205D0A9
:102A7800AA681A4B1A4002231343AB600123EA6881
:102A88001343EB602000FFF77FFF031E23D1A16DE6
:102A9800134A1140802252000A43A265E065114A98
:102AA800206D2168C262104A0263104A42631C22E8
:102AB8000A603B704A68103313434B603200019B35
:102AC800403100F0C7F903002068044A81681140CA
:102AD80004220A4382601800FEBDC046E8FFFF7F5B
:102AE800FEF0FFFF81260008592600086526000829
:102AF8000122036870B5040098689968114201D1F1
:102B0800002070BD02210842FAD105209D680540C9
:102B1800012D1ED19A68134802401143032299607F
:102B28001A60FFF779FC060023689B682B42E7D000
:102B3800FFF772FC801B0228F6D923689B682B429A
:102B4800F2D01023A26D1343A365E36D2B43E36515
:102B580006E01023A16D0B43A365E36D1A43E265FC
:102B68000120CEE7E8FFFF7F70B5060054363378C2
:102B780004000225012B26D001233370FFF7D4FE71
:102B8800051E1ED1206D831DDB7F022B08D100F0AE
:102B9800A9F9002804D040230500A26D1343A365BA
:102BA80010212268200053688B435360002D0CD1FC
:102BB800FFF79EFF051E0BD001212268D3688B43C7
:102BC800D36000233370280070BDFFF791FFF3E74F
:102BD800A26D034B1A400433FF331343A365EBE79D
:102BE800FEFEFFFF10B5FF2403220B002100024068
:102BF800D20091409B012340C943934000280ADB3F
:102C0800C0240B4A800880008018A40002590A409A
:102C18001343035110BD0F2210400838054A80089D
:102C280080008018C26911401943C161F2E7C046AB
:102C380000E100E000ED00E0002805DB1F2318405C
:102C48001E3B8340014A13607047C04600E100E024
:102C5800002809DB1F2318401E3B8340034AD36723
:102C6800BFF34F8FBFF36F8F7047C04604E100E09A
:102C78008022431E5204012093420DD2C021074AEC
:102C880007485360036A09061B021B0A0B430362C9
:102C980000200723906013607047C04610E000E0F2
:102CA80000ED00E0F0B5846CC56C6560046D002C27
:102CB80002D0446D856D65601C24056C084E254066
:102CC8001B3CAC4077683C4374600468636083686D
:102CD800102B02D1A260E160F0BDA160E260FBE7C9
:102CE8000000024010B50400036C094A9B089B18B9
:102CF8009B00436400681421C0B20838FDF70EFA3F
:102D0800044BA3641F2318401E3B8340E36410BD9B
:102D18000082001080080240F8B504000120002C51
:102D280046D02568254B1421E818FDF7F7F902234A
:102D38008000A61D2064F3772B68214AA7681340FA
:102D48002B60E36821693B430B4361692A680B43A5
:102D5800A16920000B43E1690B43216A0B4313432C
:102D68002B60FFF7BFFF8023DB019F4201D10023C7
:102D780063603F236268616C13400B60E06CA16C78
:102D8800013A4860032A14D80E4A0F4899180122BC
:102D9800013B9A40A2651300002289002165606505
:102DA8000A60436000200123E0630534F377E0778D
:102DB800F8BD002323656365A365F3E7F8FFFDBF4E
:102DC8000F80FFFF3F82001040090240F8B501253F
:102DD80004002800002C34D0276814213B68002602
:102DE800AB433B60174BF818FDF798F91C2380009C
:102DF800206418402B008340134A3E60516820002D
:102E08000B435360FFF76EFF636CE26C1E60A36CAC
:102E18005A6063685A1E032A06D895400B495B1806
:102E28009B001E600A4B5D600020A31D2065606545
:102E3800A065E06220636063A063E0630534D8772F
:102E4800E077F8BDF8FFFDBF000002403F820010A8
:102E580040090240F7B5451D0193EE7F04000220AA
:102E6800012E33D00138E877A71DFE7FB4466346AC
:102E7800F6B200960026834230D10130F8772568F3
:102E8800E6632868009B98432860019B2000FFF7B1
:102E980009FF236BB3421AD00E232A6813432B6011
:102EA800636C1A68D20304D58022196852000A4359
:102EB8001A60236D002B04D08022196852000A433F
:102EC8001A60012300202A6813432B60FEBD0422E8
:102ED8002B6893432B602A680A23DFE78023E36388
:102EE800EE77F3E7F0B5002808D0841DE37F411D95
:102EF800022B05D00423C3630023CB770120F0BD48
:102F08000E250268466C1368AB4313603368104D96
:102F18002B403360012316689E431660026C1B33F6
:102F28001A401B3B93400B4E77683B437360C26C5F
:102F3800836C5A60036D002B05D01A682A401A600A
:102F4800436D826D5A6001230020E377C877D6E786
:102F5800FFFEFFFF00000240F8B5811DCB7F022B6A
:102F680003D00423C3630120F8BD0E2402681C2784
:102F78001368456CA3431360012314689C431460D1
:102F88002A68104C22402A60026C0F4D3A40934048
:102F98006E6833436B60C26C836C5A60036D002BA0
:102FA80005D01A6822401A60436D826D5A60012369
:102FB8000022CB77431DDA77836B934200D0984782
:102FC8000020D1E7FFFEFFFF00000240F8B51C24F7
:102FD8000427016C264A21403C008C40166803688F
:102FE8001D6826420FD03D420DD01968890602D4CB
:102FF8001968B943196053681C43036B5460002B6C
:103008001BD0984719E002273C008C40264215D077
:103018003D4213D01968890606D40A251968A943C0
:1030280019600121831DD97753681C43546000221D
:10303800431DDA77C36A9342E3D1F8BD0824270019
:103048008F403E42F9D02542F7D00E251C68AC438C
:103058001C6001231D008D402900546821435160E4
:10306800821DC363D3770022431DDA77436BE2E7FF
:10307800000002400630C07FC0B27047C06B704786
:103088000020054B5A69824205DA044A9A60044ACC
:103098009A605869C00F70470020024023016745B5
:1030A800AB89EFCD8022044B120659690A435A6155
:1030B8005869C043C00F704700200240F8B50500AA
:1030C8008027FFF7A9F97F024619124C23693B4272
:1030D8000BD12269104B11001048194020611A4287
:1030E80009D00F4B0120596004E0FFF795F9B04271
:1030F800EBD30320F8BDFFF78FF980264519F602B8
:103108002369180030403342F4D0FFF785F9A8420C
:10311800F6D3EEE700200240FA830000FB830000AC
:10312800DC020020F7B5174E0193337804000D0038
:1031380002200092012B1ED00123FA2033700023B5
:1031480080007360FFF7BAFF002812D10E4F012CE0
:1031580012D17B6923437B61009B2B60BFF36F8F88
:10316800019B6B60FA208000FFF7A8FF7B69A343EF
:103178007B6100233370FEBD2800009903F044F9F9
:10318800F0E7C046DC02002000200240044A05485F
:103198005369C90003401943034B0B4353617047FC
:1031A8000020024007E0FFFF02000100F7B5214FB1
:1031B80005003B7802240191012B1AD00123FA2043
:1031C8003B70002380007B60FFF778FF041E0ED160
:1031D80004236B602B68042B0DD1FA20164A174B79
:1031E800516980000B435361FFF768FF0400002317
:1031F8003B702000FEBD0123019A5B421360AE685C
:10320800AB68EA689B18B3420CD968683100FFF7CD
:10321800BDFFFA208000FFF751FF002808D0040006
:10322800019B1E600221044A53698B435361DEE708
:103238000136E5E7DC02002000200240040001001E
:103248000023F0B585B00A681400DC4001D105B050
:10325800F0BD012514009D402C4000942A4200D165
:1032680091E04A685F0094460322644622400324A2
:10327800BC40E4430194541E012C2ED88668019C5E
:103288002640CC68BC403443846044680126AC4383
:1032980025006446240934409C402C434460C5689A
:1032A800019C25408C68BC402C43C460022A16D17E
:1032B80007250F261D40AD00AE40DC08A400041908
:1032C8000294246A03962600039CA64334000E69E0
:1032D800AE402643029C266201E0032ADFD1BA40B1
:1032E8000468019D25402A43C02402606246A40266
:1032F800224248D0254A03259C08A400A4180F227E
:103308001D40ED00AA40A027266EFF059643002227
:10331800B8420CD01E4F0132B84208D01D4F0132BE
:10332800B84204D01C4F0332B84200D1023AAA4036
:10333800674632432266154C009A2668009DD243A0
:103348003543FF0201D4350015406746256066689D
:10335800009D3543BF0201D43500154067466560BE
:103368000E4C009DE66F3543BF0301D43500154070
:103378006746E5670A4C009EE56F2E43FF0301D4BC
:1033880015402E00E66701335DE7C046001802408D
:103398000004005000080050000C005008180240BB
:1033A80004180240F0B500230F0085B03A00DA4057
:1033B80001D105B0F0BD01229A40140001923C40B1
:1033C800174253D02A4903259A08920052180F2110
:1033D8001D40ED00A940166E02910E400396A026EE
:1033E8000021F605B0420FD022498C4601216045E4
:1033F8000AD021498C460221604505D01F498C46D8
:103408000321604500D00231A940039DA94212D191
:103418001B4E1749F56FA543F5671A4EF56FA5437F
:10342800F5674D68A5434D600D68A5430D60116EA5
:10343800029CA1431166032459008C4007210F26E2
:10344800194089008E400268019922430260DA0817
:1034580092008218156AB54315628268A243826099
:1034680042688A434260C268A243C26001339DE752
:10347800001802400004005000080050000C0050E2
:10348800041802400818024000690840431E984189
:10349800C0B27047002A01D0816170478162FCE7A1
:1034A800426913000B401B0491430B43836170472F
:1034B80070B5084D0400EB68184202D0E86002F0CD
:1034C80013F92B69234203D020002C6102F0CAF9BA
:1034D80070BDC0460018024010B5114C1149236850
:1034E80002000B4003432360802300209B009A4284
:1034F8000ED10D4B0D49186806235843FCF70EFEF4
:103508008022431CD200616908001040114200D19A
:1035180010BD002B01D0013BF5E70320F8E7C046BA
:1035280000700040FFF9FFFF0000002040420F003C
:10353800F0B5040085B0002802D1012005B0F0BD27
:103548000368DB0710D423689B075CD423681B0738
:1035580000D5C1E023685B0700D5F2E0E369002BE2
:1035680000D079E10020E9E73822AF4DAB6813407D
:10357800EA68102B09D1D3439B0708D12B689B031A
:10358800E1D56368002BDED1D7E7082BF6D080227F
:1035980063685202934211D12A6813432B60FEF7E5
:1035A8003BFF80270600BF022B683B42CBD1FEF7CA
:1035B80033FF801B6428F7D90320BFE7A021C90285
:1035C8008B4208D180232968DB020B432B602B68D0
:1035D8001A432A60E3E72A6894490A402A602A685D
:1035E80093490A402A60002BD9D1FEF715FF80279E
:1035F8000600BF022B683B42A5D0FEF70DFF801BDB
:103608006428F7D9D8E73822874DAB681340EA68B1
:10361800102B28D103210A40022A26D12A685205F4
:1036280003D5E268002A00D187E7696862698148A2
:10363800120201400A436A60002B0CD12B687E4AB3
:103648007E491340226913432B602B687C4A9B04F4
:103658005B0FDA400A607B4B1868FEF795FE00287E
:1036680000D173E769E7002BD8D0E368002B20D09E
:103678002B68714A802713402269FF0013432B608F
:1036880080232A685B0013432B60FEF7C5FE060003
:103698002B683B4207D06A68636966491B020A4087
:1036A80013436B6052E7FEF7B7FE801B0228EFD981
:1036B80082E72B68644A802713402B60FEF7ACFE34
:1036C8000600FF002B683B4200D13FE7FEF7A4FE4F
:1036D800801B0228F6D96FE73822534DAB68134098
:1036E800182B08D12B6E9B0700D433E7A369002B56
:1036F80000D02FE721E7A2690123002A10D02A6E03
:10370800022713432B66FEF787FE06002B6E3B420B
:1037180000D01FE7FEF780FE801B0228F6D94BE792
:103728002A6E02279A432A66FEF776FE06002B6E5B
:103738003B4200D10EE7FEF76FFE801B0228F6D948
:103748003AE73822384DAB681340202B08D1EB6D8F
:103758009B0700D402E7A368002B00D0FEE6ECE646
:1037680080220021EB6B52050091134208D1EB6BCC
:103778001343EB63EB6B13400393039B0123009309
:103788008027324E7F0033683B4215D0A368012B57
:1037980022D1EA6D1343EB65FEF73EFE02270600D1
:1037A800EB6D3B4238D0009B012B00D0D6E6EB6B8B
:1037B800274A1340EB63D1E633683B433360FEF797
:1037C8002BFE019033683B42E0D1FEF725FE019BBA
:1037D800C01A0228F6D9EFE6EA6D052B05D1013BA0
:1037E8001343EB65EA6D0123D4E701218A43EA65B7
:1037F800EA6D03318A43EA65002BCDD1FEF70CFE52
:1038080002270600EB6D3B42CDD0FEF705FE114BBB
:10381800801B9842F6D9CFE6FEF7FEFD0D4B801BC4
:103828009842BDD9C8E6C04600100240FFFFFEFF1F
:10383800FFFFFBFFFF80FFFFFFC7FFFF0000002027
:103848000024F40008000020FFFEFFFF0070004085
:10385800FFFFFFEF8813000038213F4DAA680A4098
:10386800102A51D03D4A022B38D12B6880271340AB
:103878002B60FEF7D1FD0600BF042B683B4227D121
:10388800616A236AEA680B43354980260A40134374
:10389800E26AB6041343226B1343A26A120213436B
:1038A800EB6080232A685B0413432B608023EA685B
:1038B8005B051343EB60FEF7AFFD04002B68334252
:1038C80000D04FE6FEF7A8FD001B0228F6D973E6E4
:1038D800FEF7A2FD801B0228CFD96DE62B68802653
:1038E80013402B60FEF798FD0400B6042B683342A2
:1038F80004D1EB681B4A1340EB6033E6FEF78CFDFE
:10390800001B0228F2D957E6012B00D115E6032245
:10391800E868216A02408A4200D00EE67022616A95
:1039280002408A4200D008E6FE21A26AC90101408D
:103938001202914200D000E6F822E16A92030240A6
:103948008A4200D0F9E5236B400F4007C01A431E96
:103958009841C0B2F2E5C04600100240FFFFFFFEEA
:103968008C80C11FFCFFFEEF382370B51D4CA26888
:103978001A4205D123681C489B045B0FD84070BDD0
:10398800A2681A40082A27D0A2681A40102A17D11C
:10399800E368E168DB43E5684906490F6F322D0AA1
:1039A800013115409B0709D11048FCF7B7FBE168C6
:1039B8006843490F0131FCF7B1FBE0E70A48F4E737
:1039C800A2681A40202A09D0A26800201340182BA8
:1039D800D5D1FA20C001D2E70448D0E78020000200
:1039E800CDE7C046001002400024F40000127A001F
:1039F800F7B504000D00002801D10120FEBD0727FE
:103A08004A4E33683B408B422AD3226893073BD403
:103A1800D20748D4072733683B40AB420AD93368FA
:103A2800BB432B433360FEF7F7FC019033683B4000
:103A3800AB426BD123683E4D5B076FD4FFF794FF11
:103A4800AB683C491B051B0F9B005B581F210B40B3
:103A5800D840394A394B10601868FEF795FCCDE715
:103A68003368BB430B433360FEF7D6FC01903368E1
:103A78003B40AB42C9D0FEF7CFFC019BC01A304B8C
:103A88009842F4D90320B9E72949530704D5E0231C
:103A98008868DB0103438B608B682A480340A06871
:103AA80003438B60B4E76268214F012A19D13B6850
:103AB8009B03A2D50721BB688B431343BB60FEF76A
:103AC800ABFC01903823BA681A406368DB009A425D
:103AD800A0D0FEF7A1FC019BC01A194B9842F1D95E
:103AE800D0E7022A03D13B689B01E3D485E7002A8B
:103AF80003D13B685B05DDD47FE70223032A03D1AA
:103B0800396E1942D6D178E7F96DFAE7FEF784FCE9
:103B1800019BC01A0A4B984288D9B3E7AB680A4A96
:103B28001340E2681343AB6088E7C04600200240B8
:103B38000010024040640008000000200800002037
:103B480088130000FFF0FFFFFF8FFFFF064B0749B8
:103B58009B68074A5B045B0F9B005B581F2110683A
:103B68000B40D8407047C04600100240206400084F
:103B780000000020F0B50368050085B000209B0315
:103B880051D58022484C5205E36B0090134208D16E
:103B9800E36B1343E363E36B13400393039B01233A
:103BA80000938027414E7F0033683B433360FEF724
:103BB80033FC019033683B4227D0E16DC0220800F6
:103BC80092006B691040114217D098420CD0E36DF7
:103BD800374AE16D1340802252020A43E265E26DE2
:103BE80034490A40E265E365DB0706D5FEF714FCB5
:103BF80002270600E36D3B424ED0E36D2C4A0020BD
:103C080013406A691343E36506E0FEF705FC019B70
:103C1800C01A0228CED90320009B012B03D1E36BE5
:103C2800254A1340E3632A68D30706D503241E49AF
:103C38004B6DA3436C6823434B65930606D51A491D
:103C48001E4C4B6D2340AC6823434B6553040FD582
:103C580015492C694B6D9B009B0823434B658023BA
:103C6800DB059C4204D18023CC685B022343CB60F4
:103C780012050FD50C4A124C536DE96823400B43CB
:103C880053658023DB01994204D18023D1685B020C
:103C98000B43D36005B0F0BDFEF7BEFB094B801B9C
:103CA8009842A7D9B7E7C04600100240007000400C
:103CB800FFFCFFFFFFFFFEFFFFFFFFEFFFCFFFFF50
:103CC800FF3FFFFF881300000122036A70B593438A
:103CD8000362036A164A4468856915400A681543F1
:103CE800022293438A681343124A904205D0124E27
:103CF800B04202D0114EB04213D10826B343CE6869
:103D080033430426B343904205D00B4A904202D075
:103D18000A4A904205D10A4A8E6922404C693443C6
:103D280014434A68446085614263036270BDC046BB
:103D38008CFFFEFF002C0140004401400048014078
:103D4800FFFCFFFF036A174A70B513400362056A58
:103D5800154B4268C4691C400B681C43134B1D403B
:103D68008B681B022B43124DA8420ED1114D1D40EA
:103D7800CB681B022B43104D2B40104D4E6915404C
:103D88008A69324312012A4305E00D4DA842F4D056
:103D98000C4DA842F1D042604A68C461C263036214
:103DA80070BDC046FFFEFFFF8CFFFEFFFFFDFFFF5B
:103DB800002C0140FFF7FFFFFFFBFFFFFFCFFFFFD6
:103DC8000044014000480140036A124A30B51340DC
:103DD8000362046A104D4368C2692A400D682D02C7
:103DE80015430E4A14408A68120322430C4CA04221
:103DF80005D00C4CA04202D00B4CA04204D10B4C75
:103E08001C404B699B01234343604B68C5610364B5
:103E1800026230BDFFEFFFFFFF8CFFFEFFDFFFFFF9
:103E2800002C01400044014000480140FFBFFFFF53
:103E3800036A70B5104C114A23400362066A43684E
:103E4800456D15400A6815430D4A16408A681204E4
:103E580032430C4EB04205D00B4EB04202D00B4E4E
:103E6800B04203D11C404B691B02234343604B689B
:103E780045658365026270BDFFFFFEFF8FFFFEFF91
:103E8800FFFFFDFF002C01400044014000480140B5
:103E9800036A124A30B513400362046A104D43683E
:103EA800426D2A400D682D0215430E4A14408A6857
:103EB800120522430C4CA04205D00C4CA04202D063
:103EC8000B4CA04204D10B4C1C404B699B02234372
:103ED80043604B684565C365026230BDFFFFEFFF75
:103EE800FF8FFFFEFFFFDFFF002C01400044014071
:103EF80000480140FFFFFBFF01000300012010B54F
:103F08003D310C78E2B2844218D1001808701B6861
:103F1800D9681143D9600B498B4202D00A498B42B8
:103F28000DD19A6809490A40062A06D007398A42FB
:103F380003D0012219680A431A60002010BD1968CD
:103F4800F9E7C046002C01400004004007000100CA
:103F580070470000194A10B50368904202D0184C07
:103F6800A04208D17024A3434C68234390420BD04D
:103F7800134CA04208D0134CA04205D0124CA042CA
:103F880002D0124CA04203D1114C1C40CB682343F1
:103F98008024A3434C69234303608B68C3620B6886
:103FA8008362904205D0084B984202D0074B984252
:103FB80001D10B6903630123436110BD002C01404B
:103FC8000004004000200040004401400048014037
:103FD800FFFCFFFF70B504000120002C23D0250052
:103FE8003D352B78DAB2002B05D123003C33200075
:103FF8001A70FEF74DF802232B702068211DFFF779
:10400800A9FF2200012300204832137047340A3ADE
:10401800137053709370D370137153719371D3717C
:10402800137223702B7070BD70B504000120002C32
:1040380023D025003D352B78DAB2002B05D123009B
:104048003C3320001A70FFF783FF02232B7020688F
:10405800211DFFF77FFF2200012300204832137043
:1040680047340A3A137053709370D37013715371B5
:104078009371D371137223702B7070BD1022036A71
:1040880070B593430362056A154C426883692340FF
:104098000C6824021C4320239D438B681B012B437F
:1040A800104DA8420FD18025AB431E00CB68403D80
:1040B8001B013343AB430C4D4E6915408A693243AB
:1040C80092002A4305E0094DA842F4D0084DA842C1
:1040D800F1D042604A6884618263036270BDC04661
:1040E800FF8CFFFE002C0140FFF3FFFF004401405E
:1040F80000480140F8B507003C3715003A7803003E
:104108000C000220012A0CD0013838700C2D51D037
:1041180008D8042D2DD0082D3CD0002D17D0002311
:104128003B70F8BD102D58D0142DF8D11D6828000B
:10413800FFF7AEFE80236A6D1B0113436B656B6D41
:104148002E4A13406B6523696A6D1B0253E01D6894
:104158002800FFF7B9FD0823AA6913430422AB61BD
:10416800AB699343AB61AB6922691343AB61002030
:10417800D5E71D682800FFF781FF8023AA691B0186
:104188001343AB61AB691D4A1340AB612369AA694C
:104198001B02EAE71E683000FFF7D4FD0422F3692A
:1041A8001D43F561F3699343F361F369226913438E
:1041B800F361DCE71D682800FFF706FE8023EA6943
:1041C8001B011343EB61EB690C4A1340EB61236954
:1041D800EA691B021343EB61C9E71D682800FFF772
:1041E80027FE08236A6D134304226B656B6D9343A6
:1041F8006B656B6D226913436B65B8E7FFFBFFFFC7
:104208001F2310B5012419408C408A40036AA34338
:104218000362036A1A43026210BD000010B5082940
:104228001CD006D800290BD0042914D0030043332E
:1042380008E00C2915D01029F8D10300423301E019
:1042480003003E331B78013B5A1E9341DBB2002B1F
:104258000AD0012042E003003F33F3E70300403374
:10426800F0E703004133EDE7022308293ED009D8DF
:1042780000290ED0042932D00200433213700429D9
:10428800E7D12FE00C2939D01029F5D1423003703D
:10429800DFE702003E3213700468E2681343E3600C
:1042A800046801222000FFF7ABFF1C4A94422DD07E
:1042B8001B4B9C422AD01B4B9C4227D01A4B9C423A
:1042C80007D1A368194A1340062B06D0073A934230
:1042D80003D00123226813432360002010BD02008D
:1042E8003F32137002680423D4680DE002004032A4
:1042F80013700268D3680B43D360D1E702004132E0
:10430800137010230268D4682343F5E78023616C97
:104318001B020B4363649442D3D0CFE7002C0140C7
:10432800004401400048014000040040070001002B
:1043380010B5FFF773FF10BD30B5EFF310840122FD
:1043480082F31088C02501680B68AB430B6084F3C7
:104358001088EFF3108182F310880268044C936888
:104368002340936081F3108820238830036030BD98
:10437800FFFF7FFF30B5EFF31084012282F310882E
:104388000168134D0B682B400B6084F31088EFF322
:10439800108182F3108802680E4C93682340936062
:1043A80081F31088C36E012B0AD1EFF3108183F3D8
:1043B8001088102402681368A343136081F31088DF
:1043C800030020228C331A600023C366436730BD84
:1043D800DFFEFFFFFEFFFFEF70B505000120002D97
:1043E80019D02E0024230024883633602B681A68DD
:1043F80082431A6028001C605C609C60FDF778FFAF
:104408002B00200090331C60043B34601C60EC6679
:104418002C6784352C7070BDF7B5050088351300FE
:104428002A6804000220202A04D1002901D0002B88
:1044380001D10120FEBD8022A0685201904204D122
:104448002269002A01D1CA07F3D422002600543277
:104458002165002713805380212290363760E06F52
:104468002A6022680192B84211D0114A8763C26259
:10447800104A0263104A4263019A2832FEF7EAFCA6
:10448800B84204D010233360DB182B60D1E74022F8
:1044980023681A62EFF31081012383F310882268DE
:1044A8007F3390680343936081F310880020C1E74D
:1044B8006D450008BF450008CF450008030002000D
:1044C80080218C32883370B51B6815680268040037
:1044D80092680A4220D0212B1ED1EFF31080203B96
:1044E80083F31088226893688B43936080F3108865
:1044F800E06F00280DD0FEF7F5FC002809D0E06F2A
:10450800FEF7BCFD202804D110239034032023603B
:104518000AE02000FFF710FF402123689B680B4248
:1045280001D0222D01D0002070BDEFF310800123AF
:1045380083F31088250004CD93688B43936080F340
:104548001088E86F002808D0FEF7CCFC002804D0BB
:10455800E86FFEF793FD2028D6D02000FFF70AFF6A
:10456800E1E7704703001B6870B51A682023110043
:10457800806A19401A421AD1030056331980EFF3A2
:104588001084012282F31088802501688B68AB4370
:104598008B6084F31088EFF3108182F31088402336
:1045A800026810680343136081F3108870BDFFF739
:1045B800D8FFFBE7704710B5806AFFF7FBFF10BD17
:1045C80070477047704770B5846A230088331A684B
:1045D8005D6823689B681B0608D5212A06D123003D
:1045E8000022563320001A80FFF7A6FE23689B6836
:1045F8005B0608D5222D06D1230000225E33200059
:104608001A80FFF7B7FE22001023903211682000AD
:104618000B431360FFF7D6FF70BD806A00230200CA
:1046280010B55E321380083A1380FFF7CBFF10BD38
:1046380070470000F7B50168C14DCB6904000A68EE
:1046480088682B4210D120252B4200D19BE0802680
:10465800760515400640354300D194E0636F20008D
:10466800002B00D085E085E0B64D05400095B64D9D
:10467800009E1540354300D185E025000126903580
:10468800334205D0D70503D50E622F683E432E600E
:10469800022633420CD0C7070AD527000E6290378E
:1046A8003E680197B446042667463E43019F3E6034
:1046B800042633420CD0C7070AD527000E6290376C
:1046C8003E680197B446022667463E43019F3E6016
:1046D8000826B446334209D02027009E17403743A6
:1046E80004D066460E622F683E432E60802636014F
:1046F800334206D0570104D50E6220212E6831437B
:1047080029602968002935D020210B420AD080234E
:104718005B0511400340194304D0636F002B01D09F
:104728002000984722682B684027966828223E4038
:10473800134020001E4322D0FFF71CFE23689B680D
:104748003B4218D0EFF31081012383F31088250032
:1047580004CD9368BB43936081F31088E86F002809
:1047680009D07A4B8363FEF7F7FB002802D0E86F85
:10477800836B9847F7BD2000FFF724FFFAE7FFF7A0
:1047880021FF2E60F6E7E56E012D00D09FE0102690
:10479800334200D19BE0324200D198E00E62896832
:1047A80040230A001A40194257D0211DCA6F1068C9
:1047B800426892B2002ADDD027005C373F889742D2
:1047C800D8D927005E373A800268202084461040F6
:1047D80000906046024232D1EFF3108785F31088CB
:1047E80020685B4E02683240026087F31088EFF35E
:1047F800108785F3108820688268AA43826087F34F
:104808001088EFF3108785F31088206882689A4330
:10481800826087F31088230062468C331A60009BFD
:10482800E366EFF3108085F3108822680F3513686C
:10483800AB43136080F31088C86FFEF753FB022365
:104848002200236723005C325E331B881188C91A53
:1048580089B22000FFF7ECFE8CE7230020005C33D0
:104868005E301988038800889BB2002800D181E750
:10487800C91A89B2002900D17CE7EFF3108785F3C4
:1048880010882068334E03683340036087F310882C
:10489800EFF3108785F3108820682F4E8368334024
:1048A800836087F31088230020208C331860E26629
:1048B8006267EFF3108085F310881025226813686B
:1048C800AB43136080F3108802232367C1E7802578
:1048D8006D032B4206D0460204D520000D6200F07D
:1048E8003FFB47E780210B4207D080252D0411406C
:1048F8002840014301D0A36FB1E640210B4216D0F6
:104908000A4214D0EFF31080012383F31088226841
:1049180013688B43136080F31088230020228833A8
:104928001A6000232000A367FFF71BFE22E7190285
:1049380014D5510012D5200000F014FB1AE7C04628
:104948000F080000010000102001000423460008A1
:10495800FFFEFFFFDFFEFFFFFEFFFFEFDB0100D4DE
:1049680008E7002A00DB05E7200000F0FAFA01E773
:104978000123806A10B50367C36E012B06D10300BB
:104988005C3319884908FFF753FE10BDFFF719FE7D
:10499800FBE7000003001B6820221B6870B51900A4
:1049A800806A1140134234D103005E331980EFF35B
:1049B8001085012383F3108804681D4E2168314057
:1049C800216085F31088EFF3108583F3108804685D
:1049D800A1689943A16085F31088EFF3108483F3ED
:1049E8001088402501688B68AB438B6084F310887E
:1049F80003008C331A60C36E012B0AD1EFF31081C8
:104A080083F31088102402681368A343136081F3AA
:104A1800108800230367C36E012B05D103005C33A4
:104A28001988FFF705FE70BDFFF7CAFDFBE7C04612
:104A3800FFFEFFFF70B504002569A16803682943DC
:104A48006569C26929431868494D114328400143E3
:104A5800196059684748256A0140E0680143596070
:104A6800A16998682943444D284001430F20996063
:104A7800D96A8143606A0143D96240498B4215D1A2
:104A880003213F4B5B6D0B40013B022B60D83D4936
:104A9800C85C80231B029A422FD1082856D8FBF7FE
:104AA80033FB5B550E550B5555550F0036495B18B2
:104AB800591E8B411801ECE7FEF756FF4EE0334ACA
:104AC800616A334B49001000C95AFBF727FB656838
:104AD80040006B08C0182900FBF720FB02002D4B93
:104AE800103A9A4232D80F23020000079A4393B231
:104AF800400F22680343D36032E0082826D8FBF72A
:104B080003FB1A2505251F25252522001F48626A53
:104B18001F4B5200D15AFBF701FB65686B08C018A0
:104B28002900FBF7FBFA02001A4B103A9A420DD8FB
:104B38002368D86014E0FFF709F8002810D0E6E7EA
:104B4800FEF712FFF9E780200002E0E7012008E005
:104B580080231B029A42EED1FEF7F8FF021EAFD166
:104B680000200D4BA36600236367A36770BDC04692
:104B7800F369FFCFFFCFFFFFFFF4FF1100380140BB
:104B8800001002408064000800BCFFBF0024F4004D
:104B980084640008EFFF000001000100836A30B55B
:104BA800DA0706D50168284C4A682240C46A2243BD
:104BB8004A609A0706D50168244C4A682240046B6B
:104BC80022434A605A0706D50168214C4A682240A8
:104BD800446B22434A601A0706D501681D4C4A688F
:104BE8002240846B22434A60DA0606D501681A4CD3
:104BF8008A682240C46B22438A609A0606D50168F7
:104C0800164C8A682240046C22438A605A0610D5E2
:104C18000168134D4A68446C2A4022434A60802246
:104C28005203944205D14A680E4C2240846C2243B8
:104C38004A601B0606D502680B4953680B40C16CD5
:104C48000B43536030BDC046FFFFFDFFFFFFFEFF73
:104C5800FFFFFBFFFF7FFFFFFFEFFFFFFFDFFFFF10
:104C6800FFFFEFFFFFFF9FFFFFFFF7FFF8B504000F
:104C78000D0017001E002268D3692B405B1B5942A8
:104C88004B41BB4201D0002029E0069B0133F3D001
:104C9800FDF7C2FB069B801B984201D8002B1FD151
:104CA800EFF31080012282F310882168204D0B68F1
:104CB8002B400B6080F31088EFF3108082F310888C
:104CC80021688B6893438B6080F3108823001F3220
:104CD80088331A605A600023032084342370F8BD97
:104CE80023681A685207C6D58022D9691201114271
:104CF800C1D01A62EFF31080012282F31088216874
:104D08000B4D0B682B400B6080F31088EFF310807D
:104D180082F3108821688B6893438B6080F3108836
:104D2800220020238832136053609360D3E7C04683
:104D38005FFEFFFF030073B50026040090331E607A
:104D4800FDF76AFB236805001B681B0719D4236855
:104D58001B685B070AD58021104B002200932000B6
:104D68002B00C903FFF782FF002815D1220000207D
:104D78002023883213605360E066206784342070F3
:104D88000BE08021054B32000093890303002000CB
:104D9800FFF76CFF0028DAD0032076BDFFFFFF0184
:104DA80070B5041E01D1012070BD050088352B683F
:104DB800002B04D1020084321370FDF717FA242364
:104DC800012122682B60136820008B431360FFF7D2
:104DD80031FE0128E7D0A36A002B02D02000FFF79C
:104DE800DDFE236807495A6820000A402A215A60D4
:104DF8009A688A439A60012219680A431A60FFF781
:104E080099FFD1E7FFB7FFFFF8B5130002000600CE
:104E180005005C3281650F00138022210022903644
:104E28008C3532602960011D0400C86F904213D090
:104E38001D498263C1621D493A0001631C494163EF
:104E480021682431FEF706F8002805D01023012038
:104E58003360DB182B60F8BD2369002B0BD0EFF310
:104E68001081012383F310882268FF3310680343FD
:104E7800136081F31088EFF31080012383F3108807
:104E880021688A681A438A6080F31088EFF31081DA
:104E980083F3108822683F3390680343936081F35B
:104EA80010880020D7E7C0469D49000879490008C6
:104EB800CF45000803008C3070B504680220202C10
:104EC80025D10138002922D0002A20D080209C68D2
:104ED8004001844205D11869002802D101300142FD
:104EE80015D10020D8661868406800020CD5EFF389
:104EF8001085012080F3108880201C68C004266873
:104F08003043206085F310881800FFF77DFF70BDDF
:104F1800F7B50700436E04006A37002B04D101205F
:104F2800388068342080F7BD03680B4E9A689B6808
:104F38000A4D5B0FF05CE95CC0000192FBF778F961
:104F4800019B38801B015B0FF05CE95CC000FBF73C
:104F58006FF980B2E5E7C046A46400089C640008C5
:104F6800704770477047000070B504008434227899
:104F780003000220012A11D01D00242201268835B1
:104F88002A601A6811681068B0431060044801402C
:104F980000205866202311602B60207070BDC04629
:104FA800FFFFFFDFF8B5050084350B0029780222E2
:104FB800012915D0060001210468883622323260A2
:104FC800276822688A432260A168C900C908194372
:104FD800A160FFF79DFF20230022276033602A701D
:104FE8001000F8BDF8B5050084350A0029780223B9
:104FF800012915D006000121046888362233336060
:10500800276823688B432360A168064B1940114326
:10501800A160FFF77DFF20232760336000232B70FA
:105028001800F8BDFFFFFFF100230270FA22437158
:1050380052000B1C914200D2131CC3807047F7B575
:105048001F00490008AB1E78CBB2141E01900093D4
:1050580016D000F0CBFD009800F08AFE00F00AFEA2
:10506800451E200000F084FE00F004FE6B425D4106
:10507800013843425841EDB22D182C0000F0D8FDFC
:1050880000F0B4FD00980130C0B200F071FE00F0ED
:10509800F1FD012801D10134E4B2013EF6B2122E2D
:1050A80001D8002C05D000F0C3FD019B20001C7125
:1050B800FEBD300000F08EFE38700137EDE7F7B521
:1050C8000C001E0008AB1D780192070000F08EFD51
:1050D8006000C0B200F04CFE00F0CCFD0400019866
:1050E80000F046FE00F0C6FD01280ED1013C6342E7
:1050F8005C41013400F09CFDE0B23871FEBD3078AF
:1051080000F036FE00F0B6FD0136012CF2D0013D6C
:10511800EDB2122DF3D90024ECE7F0B503004118E5
:105128000825FF2031268B4200D1F0BD1A78504067
:105138002A0047B24400E0B2002F01DA7440E0B21E
:10514800013AD2B2002AF4D10133ECE737B54388EB
:1051580004000A339BB243800A2B5ED94279002AA5
:105168000CD10123437132330381030002320178E9
:1051780008330092AA32FFF7A2FF37BD962B4CD90D
:10518800012A4AD10223050043711C3505330178F1
:10519800002200932B00FFF752FF2379002B38D110
:1051A80006212800FFF7B9FFE31CDB7F8342E4D127
:1051B8006722237F9343182BDFD1A07F637F0002F0
:1051C800184340BAE57F80B2000228180009FBF7AF
:1051D80073FC1549FBF76EF9D6218905FBF76AF9C7
:1051E8000F2320631D40631CDB7FA21C2D02D07F90
:1051F8005B191B02C018FBF75FFC0C49FBF75AF957
:10520800D6218905FBF756F90949FBF791FA60633E
:10521800B3E7002323636363AFE7E2889A42ACD223
:10522800002363716380A8E70000C8420000484378
:10523800000048421022084B10B51B6819680A4341
:105248001A6050221A6200F0ADFFFA213822034892
:10525800C900FFF7E9FE10BD44020020F802002053
:10526800F7B5294C0121228813004800205A98429A
:1052780040D8051C904200D9151CAAB20131FA2960
:10528800F3D1934204DD214908881B189B1A0B802F
:105298001F4D2B785A1C2A70032B2AD91D4B1B4FE4
:1052A8001C881D4B05211E881C4B24B21B7836B266
:1052B8005BB201930023F85EFAF7BAFF03B218480D
:1052C80018495843FAF7B4FF0A216043FAF7B0FFC8
:1052D800019B80195843144B144A00B21880117866
:1052E800012909D11B88124A1BB2138000233B8075
:1052F8002B70F7BD0300C1E71278002AF6D11B888E
:105308000C4A1BB2F1E7C046700300203A030020A4
:1053180039030020660300206403002028000020D1
:10532800E40C0000FF0F00006E030020660500205B
:105338006C0300206A030020F0B50825012602004E
:105348000B4F0C4801390B4B89B2994200D1F0BD83
:10535800137858402B0004004008344001D07840AE
:1053680080B2013BDBB2002BF5D10132EAE7C0463F
:1053780001A0FFFFFFFF0000002130B58BB00C2219
:1053880007A8069100F0FCFF02230293DB180393A1
:105398000B3304930125274B06AC1A881B8822700F
:1053A8001B0A6370244B05951A881B88A2701B0A78
:1053B800E370224B1A881B8822711BB21B1263717F
:1053C8001F4B1A881B88A2711BB21B12E3711D4B5D
:1053D8001A881B8822721BB21B1263721A4B1A8816
:1053E800A2721B881BB21B12E372184B1B88A38185
:1053F800FDF746FE01A902A8FDF7D8FE002802D055
:10540800FDF750FE0AE02800069A079B1049FDF7B1
:1054180089FE002805D0FDF745FE032528000BB0BE
:1054280030BD2800089A099B0A49FDF77BFE051E36
:10543800E6D0F0E76405002068030020660300203A
:10544800640300205E030020240000205A0300208B
:10545800007800080878000810B5012383F3108845
:10546800FFF78AFF002383F3108810BD022330B5AD
:10547800012487B0154D0293DB1803930A33049374
:105488002B68059408332B60FDF7FAFD104B2A684A
:105498009A420AD90F4B01A902A82B60FDF786FE94
:1054A800002802D0FDF7FEFD0CE00B4B01201A8806
:1054B8002968002392B2FDF735FE041EF2D0FDF7ED
:1054C800F1FD0324200007B030BDC04620000020B5
:1054D800D8770008007000086203002010B50400A7
:1054E800A02001222021C005FDF7D4FF2200094990
:1054F8000948FEF791FF0948FDF7BCFD0128FAD1DC
:10550800043000F003FFA02000222021C005FDF791
:10551800C1FF10BDE7050020440200208C010020D7
:10552800F0B55F4C85B0E378A2781B021343677926
:1055380003935EBA2379062120003F021F43FFF739
:10554800FBFE030ADBB20193C3B20293554B7DBA4B
:105558001A88554BB6B25A80544AADB2127852B234
:105568009A80534A1278DA80524A12881A81524A2B
:1055780012885A81514A12889A81514A1288DA81CE
:10558800504A12881A82504A1178504A09021278F1
:105598000A435A824E4A12889A824E4A1288DA82FE
:1055A8004D4A12881A8372190C2A55DCA27902997D
:1055B8008A4272D1E27901998A426ED1474F2278A4
:1055C80076003A706278F61800243B007A706A0018
:1055D800BA70E8B20233844235D16400E4B2E11C07
:1055E8003800C9B2FFF7A8FE6B00FB18D870AB1CD7
:1055F800000A5B000534F854E0B2FFF76FFFFE23A2
:10560800039A1B029A4248D1254B02999A798A42F9
:1056180043D1DA7901998A423FD1304C1A78052171
:1056280022705B782E4A6370138820001B0AE3708F
:1056380013886D00A5702371FFF77EFE6071000A64
:10564800A071072027E00021725E01341112597001
:105658009A70E4B20236BDE7FF23039A1B029A420E
:10566800CDD180235B009F4217D1A379029A934240
:1056780013D1E379019A93420FD10024194D174EA3
:1056880003E02B5D33550134E4B22800FAF734FD0A
:105698008442F6D3C0B2FFF721FF05B0F0BDC04683
:1056A800670500206E0300203C030020270000202F
:1056B8002600002068030020660300206403002001
:1056C800620300205E0300205C0300205D030020CD
:1056D800240000205A03002058030020E70500207A
:1056E800600300200C000020F7B50400A020402132
:1056F800C005FDF7C9FE4B4B80211870A020C005DE
:105708000193FDF7C1FE802C38D1012831D1FCF777
:1057180083FE454E05003368C31A072B0FD8FA21BC
:105728000420890000F0B4FD404F3B78012B06D1DE
:10573800FA210220490000F0ABFD00233B70019BD9
:1057480035601B78012B03D1394A13780133137064
:10575800384A13780133DBB21370092B09D9344B5B
:1057680035491878022807D90120087000211170DE
:105778001970324BDC60F7BDFF20F6E7082CF8D132
:1057880003202F4900F084FDA0202100C005FDF76B
:105798007BFE0128EDD12B4B2B4E2C4D2C4918703C
:1057A8002B880A88378812B21BB23FB29B1A294E3F
:1057B800294ABB4226DD0020337810700133DBB262
:1057C8003370022B05D9254A1070FA2B01D903230F
:1057D8003370234B00229A5E092ACADD2B881BB23C
:1057E800D8171B1843409BB29342C2DA0B881BB2EE
:1057F800D9175B184B409BB29A42BADD0022174B6F
:105808001A70B6E70027137837700133DBB21370CC
:10581800022BDED9114E3070FA2BDAD9032313701C
:10582800D7E7C046380300203403002026000020B4
:105838003303002032030020280000200018024013
:105848008813000066050020240000206C03002057
:105858006A030020310300203003002027000020C5
:105868005A030020010010B5082807D1A020C00560
:10587800FDF70AFE002801D1014B187010BDC04683
:105888006605002070B5214C05002000FEF7A4FD38
:10589800012D37D0023D6B425D411D4B68421840D7
:1058A80096239B01C0181B4B0C22236000236060C9
:1058B8002000A360E36023616261A361E361236266
:1058C8006362A362FFF76CFA002801D0FCF76AFB59
:1058D80000212000FFF766FB002801D0FCF762FBDF
:1058E80000212000FFF77EFB002801D0FCF75AFBBF
:1058F8002000FFF739FB002801D0FCF753FBFFF726
:1059080099FC70BD9620C001CDE7C0464402002036
:1059180080BB000000380140F7B5904C062165793E
:1059280023792D021D436DBAE778ABB20193A378B2
:1059380020003F021F43FFF7FFFC0600884B0622AA
:1059480018002100019300F047FD019AF3B2360ACE
:10595800F6B29371D671F0221201974229D1A27939
:105968009A4214D1E379B34211D1ABB2013BF62B81
:1059780011D87C4F3E883D80B6B2FFF76DFD0028F8
:1059880006D16378002B02D00820FFF7A7FDF7BDEA
:10599800F6B23E80FBE7FF23019A0621200013712F
:1059A8005371FFF7C9FC019B9871000AD8712378DD
:1059B800E8E78022D20097421BD1A2799A42E6D129
:1059C800E379B342E3D1FA23AAB29B009A42DED824
:1059D800654E34883580A4B2FFF73EFD002854D1C7
:1059E8000830FFF77BFD614A338812689BB2536326
:1059F800CDE7A0212AB2C9008F4228D1A1799942C6
:105A0800C5D1E379B342C2D15948ABB21B18594941
:105A18009BB28B42BBD80A20574B584C5043268820
:105A2800198836B209B2FAF703FCABB200B2053BEB
:105A380020800F2B00D8258023881BB2042BA6DDDD
:105A480023881BB2142BA2DCFFF706FD37E0C02227
:105A5800D20097421BD1A2799A4200D097E7E37906
:105A6800B34200D093E7424AABB29446414A6344FA
:105A78009BB2434E934200D989E73488358024B2DB
:105A8800FFF7EAFC002800D17EE734807FE7E022B8
:105A9800D200974218D1A2799A4200D077E7E379E9
:105AA800B34200D073E7374B374A384C1A600022AC
:105AB8002688374B2580B6B21A80FFF7D7FC002816
:105AC80000D161E7268062E78022120197421BD14C
:105AD800A2799A4200D05AE7E379B34200D056E758
:105AE800ABB2032B00D952E72A4E3488358024B252
:105AF800FFF7B2FC0028C8D10830FFF7EFFC308868
:105B080000B2FFF7BFFE42E7A022120197420ED172
:105B1800A2799A4200D03AE7E379B34200D036E757
:105B28001D4BAAB29A4200D931E71C4EA5E7B02214
:105B38001201974200D02AE7A2799A4200D026E7BC
:105B4800E379B34200D022E7134BAAB29A4200D9B4
:105B58001DE7134C0023E65E258075E767050020E6
:105B6800E7050020640500206803002040010020AC
:105B7800E40C0000C81900006E0300206603002032
:105B88006403002020000020D8770008620300206A
:105B9800600300205E030020DC05000024000020D4
:105BA8005A03002010B50E4B0E491A7809888A420C
:105BB8000ED10D49097808290AD15B78032B04D046
:105BC800062B04D1FFF7A8FE01E0FFF7A9FC10BDE2
:105BD800002AFCD1044A1278082AF8D15B78EFE74A
:105BE8006705002064050020E706002070B58026C0
:105BF800A0248025E405760131002D012000012232
:105C0800FDF748FC290001222000FDF743FC042091
:105C180000F094FB310000222000FDF73BFC04203B
:105C280000F08CFB290000222000FDF733FC70BD3A
:105C380070B58026A0248025E405360131006D0169
:105C480020000022FDF726FC290000222000FDF795
:105C580021FC042000F072FB310020000122FDF736
:105C680019FC290001222000FDF714FC042000F093
:105C780065FB70BD8021A02070B501224901C005D7
:105C8800FDF708FC012000F059FB8021A02001222B
:105C98000901C005FDF7FEFB8026012000F04EFB40
:105CA80065257601A0203100C005FDF7EDFB041E37
:105CB80007D102008021A0200901C005FDF7EAFBF9
:105CC80006E0013DEDB2002DECD1FFF7B1FF012454
:105CD800200070BD70B58025A0248026E4052D0124
:105CE8002900760120000022FDF7D4FB31000022B4
:105CF8002000FDF7CFFB022000F020FB2900012245
:105D08002000FDF7C7FB022000F018FB2900200047
:105D18000022FDF7BFFB310001222000FDF7BAFB8E
:105D280070BD70B58025A0248026E4052D012900CA
:105D3800760120000022FDF7ADFB31000122200092
:105D4800FDF7A8FB042000F0F9FA29000122200041
:105D5800FDF7A0FB042000F0F1FA29002000002242
:105D6800FDF798FB310001222000FDF793FB70BD81
:105D7800F8B580210400A0200022A0268027090170
:105D8800C005FDF787FB0825F6053F0163B2012230
:105D9800002B00DB0022802130004901FDF77AFB4F
:105DA800022000F0CBFA012239003000FDF772FB27
:105DB800022000F0C3FA013D002239003000FDF74F
:105DC80069FB64000220EDB200F0B8FAE4B2002DDD
:105DD800DCD1F8BDF7B58027A0260825002401905E
:105DE8003F01F605002239003000FDF753FB022081
:105DF80000F0A4FA390030000122FDF74BFB8021A6
:105E0800640030004901E4B2FDF73EFB002801D0F0
:105E18000134E4B2013D0120EDB200F08FFA002D0B
:105E2800E0D1019B002B03D1FFF77BFF2000FEBDD3
:105E3800FFF750FFFAE70000F7B5FFF7FBF9B24BA1
:105E48001A88B24B1A801A88002A03D01988B04AD7
:105E5800914201D101221A80AE4B1A88AE4B1A80AA
:105E68001A88002A03D01988A94A914202D1AF2280
:105E780092001A80A94C1B8822689BB25363A84BD6
:105E880000229A5EA74B1A801A88002A03D01A8823
:105E980012B2013201D10A221A80A34B00229A5E63
:105EA800A24B1A801A88002A03D01A8812B201322B
:105EB80001D100221A809E4B00229A5E9D4B1A80C7
:105EC8001A88002A03D01A8812B2013201D100229E
:105ED8001A80188800B2FFF7D5FC974B00229A5E0B
:105EE800964B1A801A88002A03D01A8812B20132F7
:105EF80001D128221A80924B00229B5E5A1C92B232
:105F0800012A00D800238F4A814913808C46002239
:105F18008D488E4B8E4E03601F00198808373180DC
:105F2800358819890097002D02D03588654501D13B
:105F3800002535804D1E874FADB2BD4200D90021E6
:105F480035888D4200D2C5E0002A00D003602000C9
:105F5800FDF7D2FF00212000FEF7EAF97E4C200071
:105F6800FEF7ACFA802220007C49FEF7A3FF7C4BA9
:105F7800FA2201937B4B019918000093FCF760FD0E
:105F8800A02000222021C005FDF784FA322100203C
:105F980000F07EF9FA210120490000F079F9032088
:105FA800714900F075F9FA210420890000F070F9B0
:105FB8000A21052000F06CF90024002000F092F975
:105FC800002809D00098FCF7CFFDFFF749F9FA221D
:105FD80001990098FCF734FD012000F083F90028AE
:105FE80006D00022614B012161481A80FDF758FA5A
:105FF800022000F077F9002833D0A0200421C00542
:10600800FDF74EFAE1230134A4B25B019C4228D982
:10601800338801339BB2338032883D4B9A4201D199
:1060280000233380534B1F78534B1878FBF7DCFC65
:1060380004000D001E2F5AD83800FBF7D5FC4F4A34
:106048004F4BFBF709FA22002B00FAF7FDF900285D
:1060580004D04C4A138801339BB21380FFF706FA29
:106068000024032000F03EF9002802D00222464B0B
:106078001A70042000F036F900280BD0022000F036
:106088001DF9A02001220421C005FDF703FA012211
:106098003E4B1A70052000F025F9002810D03C4D21
:1060A8002800FFF753F86B79022B09D1286BFAF710
:1060B800E9F9314F3870686BFAF7E4F92D4F387009
:1060C800344D2B78002B00D177E7FFF76BFD0023C9
:1060D8002B7072E7304B009D9D4203D02B000122AC
:1060E800318019E7002A00D131E72C4B2EE778429E
:1060F800FBF77AFC214A224BFBF7AEF90022284B2A
:10610800FAF71CFD9FE7C0460078000864050020E8
:10611800FFFF00000278000868030020400100200B
:10612800047800086603002006780008640300204D
:10613800087800085E0300200A7800082400002080
:106148000C7800085A030020200000200070000886
:1061580062030020FDFF00004402002067060020C3
:1061680070030020DC000020881300005603002084
:10617800000400505D0300205C030020CDCCCCCC93
:10618800CCCC064060030020270000202600002019
:10619800F8020020E7060020E0770008D87700081A
:1061A80000806640002370B50C251C0012492800A9
:1061B800584301330A1854609460547044540A2BAD
:1061C800F5D1FA210D4B89001868F9F7A7FF80234C
:1061D80001385B0498420DD2C021094A0906506073
:1061E8000848036A1B021B0A0B43036207239460D7
:1061F800136070BDFEE7C046F006002000000020D6
:1062080010E000E000ED00E01B4A70B51368002BB9
:1062180007D01368013B1360002B02D10122174BF2
:106228001A7000220C25012615482C005443031926
:10623800596800290AD0596801395960002905D1DF
:106248005E70215C012901D19968596001320A2ADE
:10625800EBD10C4B1A6801321A6019680A4A91424C
:1062680001D100221A60094A13780133DBB2092BE5
:1062780000D90023137070BD6C0700206807002048
:10628800F0060020EC060020FFFFFF7FE806002054
:10629800020010B5092800D9FEE7012484F310880C
:1062A8000C205043044B1A18516091600021517022
:1062B800C45481F3108810BDF0060020030009289B
:1062C80000D9FEE7012282F310880C2058430023EE
:1062D800034A11184B604B70835483F3108870473E
:1062E800F006002002000020092A09D80C214A43A0
:1062F800054B9B1859780022C8B2012901D15A7060
:1063080070471000FCE7C046F006002000280FD0B8
:10631800012800D10130012383F310880022054BA6
:106328001860054B1A7082F310881A78012AFCD17C
:106338007047C0466C070020680700200D4B70B5F9
:106348000D4906001868F9F7E9FE00230B4C46438F
:106358006568A168A2689142FCD006D95B189B1AAF
:10636800B34200D370BD1100F4E7A81AC318CB18C4
:10637800F6E7C0460000002040420F0010E000E0B1
:1063880003008218934200D1704719700133F9E76E
:1063980070B500260C4C0D4D641BA410A64209D103
:1063A800002600F023F80A4C0A4D641BA410A642EC
:1063B80005D170BDB300EB5898470136EEE7B3003E
:1063C800EB5898470136F2E7AC640008AC64000863
:1063D800B0640008AC640008002310B59A4200D1EC
:1063E80010BDCC5CC4540133F8E70000F8B5C046D2
:1063F800F8BC08BC9E467047F8B5C046F8BC08BC57
:106408009E4670470000000001B40248844601BC63
:08641800604700BF2D000020C9
:10642000000000000000000000000000000000006C
:106430000100000002000000030000000400000052
:10644000000000000000000000000000000000004C
:10645000000000000000000000000000000000003C
:106460000100000002000000030000000400000022
:1064700006000000070000000800000009000000FE
:1064800004020800010002000400060008000A00DF
:106490000C001000200040008000000108040204ED
:0C64A000080101010101010307010000D7
:0464AC00E100000803
:0464B000B900000827
:1064B4000024F40001000000040000004443452DC2
:1064C400323430332D56352E322E315F48414C0054
:1064D40000700008280001010100000080220C4B1C
:1064E40030B55C69D20222435A61EFF3108272B66E
:1064F4004C1CFF34401A0D68455004318C42FAD1CB
:106504008021490218690842FCD182F3108830BD09
:046514000020024021
:040000050800233D8F
:00000001FF
